:020000040000FA
:020000000828CE
:020008000900ED
:10001000203084008001840A60300402031C0A2816
:100020002A16FF30C20041148316850185158312FC
:10003000850107309900C03083168100831231306A
:1000400090008E018F0100308B00003083168C00F1
:100050008312831631309B001C141A088312C500CA
:1000600017304502031C3528C50164000000D30B7E
:100070004F28851940280A30C207031847284F28FF
:1000800041184F280A30C202031C4B284F28411048
:10009000FF30C2004F284114C20162214F288F084F
:1000A000031935288F0100304502031D60283F10D9
:1000B000BF10BF123F137921D521E8210322162258
:1000C00001304502031D6D283F10BF10BF123F13C2
:1000D0007921D521E8213E22162202304502031D56
:1000E0007A283F10BF10BF123F137921D521E82194
:1000F0000322892203304502031D87283F10BF10C9
:10010000BF123F137921D521E8213E2289220430F4
:100110004502031D94283F10BF10BF163F177921D9
:10012000D521E8210322162205304502031DA1280E
:100130003F10BF10BF163F177921D521E8213E227D
:10014000162206304502031DAE283F10BF10BF1611
:100150003F177921D521E821032289220730450262
:10016000031DBB283F10BF10BF163F177921D521B3
:10017000E8213E22892208304502031DC7283F108E
:10018000BF10BF163F177921D521562216220930FC
:100190004502031DD3283F10BF10BF163F1779211A
:1001A000D521562229220A304502031DDE283F149C
:1001B000BF10BF163F177921562216220B30450279
:1001C000031DE9283F14BF10BF163F17792156229F
:1001D00029220C304502031DF5283F14BF10BF161D
:1001E0003F177921E821032216220D304502031D15
:1001F00001293F14BF10BF163F177921E8213E2285
:1002000016220E304502031D0D293F14BF10BF16E4
:100210003F177921E821032289220F304502031D6F
:1002200019293F14BF10BF163F177921E8213E223C
:10023000892210304502031D24293F14BF14BF1624
:100240003F177921E821162211304502031D2F297D
:100250003F14BF14BF163F177921E821292212301D
:100260004502031D3A293F14BF14BF163F177921D9
:10027000E821892213304502031D3F29B3211430A0
:100280004502031D4A293F14BF14BF163F1794218E
:100290000322162215304502031D54293F14BF14B2
:1002A000BF163F179421472216304502031D6129CE
:1002B0003F10BF10BF163F137921D521E82103223B
:1002C00016223528C50A173045020318C5018B13BD
:1002D000450883161C159A0031309B0055309D004F
:1002E000AA309D009C149C1873291C1183128B1733
:1002F0000800B00A0A303002031C0800B11C851245
:10030000B1180512FA30311C2D303002031C0800E0
:10031000B10A3F1CB1100130BF1EB100B11C8516DF
:10032000B1180516B0010800B00A0A303002031CEB
:1003300008008512051205111E30B11864303119FC
:100340008C303002031C08000310B10DB1193114B8
:10035000B1080319311431188516B1180516311971
:100360000515B0010800B00A0A303002031C08006D
:10037000851205120511851005107D30311C533092
:100380003002031C0800B10A0330B105B10803199B
:10039000851603190516B1180515B11885143118FD
:1003A000D329B1180514B0010800B20A0A3032028C
:1003B000031C08000512FF30331C37303202031CC7
:1003C0000800B30A01303F1FB3000516B201080050
:1003D000B40A0A303402031C0800B51C0511B51814
:1003E0008510F630351C32303402031C0800B50A83
:1003F000BF1CB51001303F1FB500B51C0515B51861
:100400008514B4010800B60A0A303602031C08003D
:100410008510F030381C1E303602031C0800B80A64
:1004200001303F1FB8008514B6010800B90A0A3030
:100430003902031C08000510F3303A1C2830390239
:10044000031C0800BA0A01303F1FBA000514B901A5
:100450000800B90A14303A1C46303902031C08005F
:10046000051064303A1C6E303902031C0800BA0AC9
:1004700001303F1FBA000514B90108003608B60B59
:1004800008000508023A8500C830B60008003608A2
:10049000B60B0800B70A371C08000508023A8500A9
:1004A0000510851C0514A030B6000800A80F5E2AB0
:1004B000A80A0310AA0DAA1AAA15AA12FC22AB00B8
:1004C0001330AA19AB0268302A050319692A85106E
:1004D00005152A132B080E020318742A14302A0556
:1004E0000319742A851405118F08031D0800640080
:1004F0002B080E02031C742A14302A050319822AC1
:100500008510051528302A050319882A8514051138
:100510000800A80F912AA80A0310AA0DAA1AAA1562
:10052000AA12FC22AB001330AA19AB0268302A05CC
:10053000031D05102A132B080E020318A32A1430DA
:100540002A05031D05148F08031D080064002B08ED
:100550000E02031CA32A14302A05031D051028309F
:080560002A05031D0514080023
:0805F80003308A00280382078A
:10060000143417341B341E342134253428342B344D
:100610002E343134343437343A343D344034423477
:10062000453448344B344D345034523455345734B7
:100630005A345C345F3461346334663468346A3409
:100640006C346F34713473347534773479347B346B
:100650007D347F34813483348434863488348A34DE
:100660008C348D348F34913492349434963497345E
:1006700099349A349C349D349F34A034A234A334EA
:10068000A434A634A734A834AA34AB34AC34AE3482
:10069000AF34B034B134B234B434B534B634B73422
:1006A000B834B934BA34BB34BC34BD34BE34BF34CE
:1006B000C034C134C234C334C434C534C634C7347E
:1006C000C834C934CA34CA34CB34CC34CD34CE3433
:1006D000CE34CF34D034D134D134D234D334D434F2
:1006E000D434D534D634D634D734D834D834D934B5
:1006F000DA34DA34DB34DB34DC34DD34DD34DE347C
:10070000DE34DF34DF34E034E034E134E134E23449
:10071000E234E334E334E434E434E534E534E63419
:10072000E634E734E734E734E834E834E934E934EC
:10073000EA34EA34EA34EB34EB34EB34EC34EC34C2
:10074000EC34ED34ED34EE34EE34EE34EF34EF349B
:10075000EF34EF34F034F034F034F134F134F13478
:10076000F134F234F234F234F334F334F334F33456
:10077000F434F434F434F434F534F534F534F53435
:10078000F534F634F634F634F634F734F734F73417
:10079000F734F734F834F834F834F834F834F834FB
:1007A000F934F934F934F934F934FA34FA34FA34DE
:1007B000FA34FA34FA34FA34FB34FB34FB34FB34C5
:1007C000FB34FB34FB34FC34FC34FC34FC34FC34AC
:1007D000FC34FC34FC34FD34FD34FD34FD34FD3494
:1007E000FD34FD34FD34FE34FE34FE34FE34FE347C
:0E07F000FE34FE34FE34FE34FE34FF34FF349B
:084000000000010001000100B5
:02400E00CC01E3
:00000001FF
